S01E000074696E794B32325F4B424F4F545F6C65645F64656D6F2E737265631D
S113C0008808FF1FD9C4000045C5000045C50000CD
S113C01045C5000045C5000045C5000000000000FE
S113C02000000000000000000000000045C5000002
S113C03045C500000000000045C50000F9C8000027
S113C04045C5000045C5000045C5000045C50000C4
S113C05045C5000045C5000045C5000045C50000B4
S113C06045C5000045C5000045C5000045C50000A4
S113C07045C5000045C5000045C5000045C5000094
S113C3C06B636667FFFFFFFFFFFFFFFFFFFFFFFFDA
S113C3D0FFFF8813FFFFFFFFFFFFFFFFFFFFFFFFCC
S113C3E0FFFFFFFFFFFFFFFFFFFFFFFFFFFFFFFF59
S113C3F0FFFFFFFFFFFFFFFFFFFFFFFFFFFFFFFF49
S113C400FFFFFFFFFFFFFFFFFFFFFFFFFEFFFFFF39
S113C41010B5054C237833B9044B13B10448AFF37A
S113C42000800123237010BD6804FF1F000000007A
S113C4309CC9000008B5064B1BB106480649AFF37A
S113C44000800648036813B1054B03B1984708BD43
S113C450000000009CC900006C04FF1F6404FF1F5F
S113C46000000000154B002B08BF134B9D46A3F59D
S113C470803A00218B460F461348144A121A00F0E2
S113C4807FFA0F4B002B00D098470E4B002B00D0A7
S113C49098470020002104000D000D48002802D018
S113C4A00C48AFF3008000F045FA2000290000F0AA
S113C4B081F900F02BFA00BF000008008808FF1F74
S113C4C000000000000000006804FF1F8804FF1F34
S113C4D0000000000000000072B60E480E4988609B
S113C4E00E4A0E4B0D4C0D4D0C4E0C4FB846B94632
S113C4F0BA46BB46BC460A4885460A4880470A48AD
S113C50080470A48804762B604480449084A90476D
S113C510FFF7FEBF00C0000000ED00E000000000D7
S113C5208808FF1FADC6000009C600009DC60000B4
S113C530B5C7000072B600F0B9F800F065F862B64D
S113C540FFF790FFFFF7FEBF80B400AF154B4FF02D
S113C550FF32C3F88020134B4FF0FF32C3F884201E
S113C560104B4FF0FF32C3F888200E4B4FF0FF32D0
S113C570C3F88C200B4B4FF0FF32C3F89020094BCB
S113C5804FF0FF32C3F89420064B4FF0FF32C3F84C
S113C5909820044B4FF0FF32C3F89C20BD465DF851
S113C5A0047B704700E100E080B400AF154B4FF00E
S113C5B0FF32C3F88021134B4FF0FF32C3F88421BC
S113C5C0104B4FF0FF32C3F888210E4B4FF0FF326F
S113C5D0C3F88C210B4B4FF0FF32C3F89021094B69
S113C5E04FF0FF32C3F89421064B4FF0FF32C3F8EB
S113C5F09821044B4FF0FF32C3F89C21BD465DF8EF
S113C600047B704700E100E080B487B000AF1C4BAE
S113C6101C4A9A601C4B7B611C4B3B611C4B7B602E
S113C6207A683B69D31ABB607A693B699A420ED037
S113C6300AE07B695A1C7A613A69511C39611278A3
S113C6401A70BB68013BBB60BB68002BF1D1114B76
S113C650FB60114B3B603A68FB68D31ABB6007E090
S113C660FB685A1CFA6000221A70BB68013BBB606D
S113C670BB68002BF4D11C37BD465DF8047B7047C2
S113C68000ED00E000C000000004FF1FC4C900006A
S113C6902CCA00006804FF1F8804FF1F80B500AF88
S113C6A0FFF752FFFFF780FF80BD00BF80B400AFEB
S113C6B00B4B0B4AD2F8882042F47002C3F888204E
S113C6C0084B4CF22052DA81064B4DF62812DA81DF
S113C6D0044B4FF4E9721A80BD465DF8047B704741
S113C6E000ED00E00020054080B483B000AF1A499B
S113C6F0194B03F5815318331B6843F4785201F541
S113C700815318331A601449134B03F580530433CF
S113C7101B6843F4403201F5805304331A6000234C
S113C720FB7111E00D4B02224FF4807143F822108B
S113C7300B4B0B4A51690222012000FA02F20A4310
S113C7405A61FB790133FB71FB79002BEAD00C377A
S113C750BD465DF8047B70470070044000B004409F
S113C76080F00F4080B483B000AF7860064B064A77
S113C770D1680222012000FA02F20A43DA600C377F
S113C780BD465DF8047B704780F00F4080B483B0F1
S113C79000AF7860064B064A51680222012000FA75
S113C7A002F20A435A600C37BD465DF8047B7047B9
S113C7B080F00F4080B500AFFFF796FF00F080F8DF
S113C7C00020FFF7E3FF0020FFF7CCFF4FF47A705F
S113C7D000F082F8F7E700BF80B483B000AF0346EF
S113C7E03960FB7197F90730002B0BDA0D49FB799F
S113C7F003F00F03043B3A68D2B21201D2B20B44E5
S113C8001A7609E0084997F907303A68D2B212015A
S113C810D2B20B4483F800230C37BD465DF8047B89
S113C820704700BF00ED00E000E100E080B582B099
S113C83000AF78607B68013BB3F1807F01D30123B3
S113C8400FE00A4B7A68013A5A604FF0FF300F212B
S113C850FFF7C2FF054B00229A60044B07221A60BF
S113C860002318460837BD4680BD00BF10E000E035
S113C87080B400AF034B1B681846BD465DF8047BCB
S113C880704700BF8404FF1F80B483B000AF78609A
S113C890034B7A681A600C37BD465DF8047B704719
S113C8A08404FF1F80B400AF044B1B685A1E034B63
S113C8B01A60BD465DF8047B704700BF8404FF1F07
S113C8C080B500AF034B1B689B0A1846FFF7AEFF09
S113C8D080BD00BF0004FF1F80B582B000AF786048
S113C8E07868FFF7D1FF00BFFFF7C2FF0346002BB4
S113C8F0FAD10837BD4680BD80B500AFFFF7B8FF59
S113C9000346002B01D0FFF7CDFF80BD08B5074BD0
S113C910044613B10021AFF30080054B1868836A05
S113C92003B19847204600F033F800BF0000000030
S113C93098C9000070B50E4B0E4DED1AAD100024D1
S113C9401E46AC4204D056F8242090470134F8E740
S113C95000F024F8084D094BED1AAD1000241E46D2
S113C960AC4204D056F8242090470134F8E770BD57
S113C970BCC90000BCC90000C0C90000BCC900009B
S113C98002440346934202D003F8011BFAE77047BE
S113C990FEE700BF430000000404FF1FF8B500BF1A
S113C9A0F8BC08BC9E467047F8B500BFF8BC08BC8C
S107C9B09E467047E4
S10BC9B4B0FAFF7F010000004E
S107C9BC35C400007A
S107C9C011C400009A
S113C9C4000040010000000000000000000000001E
S113C9D4000000000000000000000000000000004F
S113C9E40000000094C900000000000000000000E2
S113C9F4000000000000000000000000000000002F
S113CA04000000000000000000000000000000001E
S113CA14000000000000000000000000000000000E
S10BCA24000000000000000006
S903C4D95F
